:100000000C9401020C9429020C9429020C942902EC
:100010000C9429020C9429020C9429020C942902B4
:100020000C9429020C9429020C9429020C9442127B
:100030000C9429020C9429020C9429020C94290294
:100040000C9460130C9429020C9429020C9429023C
:100050000C9429020C9429020C9429020C94290274
:100060000C9429020C942902526573756D65005138
:100070007569740068006F0053696E676C65207065
:100080006C617965722067616D65004D756C74698E
:10009000706C617965722067616D65004F7074697D
:1000A0006F6E730078008B009C00506F636B6574FB
:1000B00020456D70697265730003053F213F12088A
:1000C000120A100A0E1C0E0C1E0C141A14161F16FF
:1000D0001E131E1E1B1E1E1F1E3F213F3A2F3A17C6
:1000E0003D173F213F181F02040A041F0E04040E8F
:1000F0001F0A1F0A0E0E1F04110E2E252E2F2A2E48
:10010000262929021F02081F08150E04040E150EC9
:1001100015151B151B040604040C04000000001731
:10012000000300031F0A1F16371A1904130A153A91
:10013000000300000E11110E000A040A040E040050
:1001400030000404040010001804031F111F121FC4
:10015000101D151711151F07041F17151D1F151D3D
:1001600001011F1F151F17151F000A000032000490
:100170000A110A0A0A110A040115020E11171E05B6
:100180001E1F150A0E110A1F110E1F15111F050142
:100190000E111D1F041F111F1108100F1F041B1F1C
:1001A00010101F061F1E040F0E110E1F09060E1140
:1001B0002E1F051A121509011F011F101F0F180FFE
:1001C0001F0C1F1B041B031C03191513001F110315
:1001D0000418111F000201022020200001020C124D
:1001E0001E1F120C0C12120C121F0C1A14041E05E6
:1001F000242A1E1F021C141D1020201D1F0814116C
:100200001F101E041E1E021C0C120C3E0A040C12AF
:100210003E1E040214160A020F120E101E0E100EBD
:100220001E081E120C1226281E322A26041E210029
:100230001F00211E040102013F213F0A4E6F20537F
:10024000442063617264206F720A6E6F204C4F41CC
:100250004445522E4845580A0A153A4578697400B3
:100260001D20466C617368696E670A20206C6F619F
:100270006465722E2E2E0A0A444F4E275420545580
:10028000524E204F464621000A0A153A49676E6FC2
:100290007265006D560A0A504C454153452054552D
:1002A000524E204F464620004C4F57204241545456
:1002B0004552592120001753440016137800161395
:1002C00014001510200015201000540A03E1818647
:1002D0007F3E186D830F0F0E0183866033186DC348
:1002E000198F1803C38E6033186DE330CF1803C322
:1002F0009E603630CDE360CF3006C79E7E3E30CD67
:10030000B360CF300CC6F6603330D9B660CF33CF90
:10031000CCF66061B0DB1E60CF30D86CE6C061B057
:10032000DB1E618F19986CC6C063B19B0E330F0F33
:10033000B078C6FF7E1F1B061E0F0500893008021D
:100340003802497868140000F6E8DBCFC3B8AEA4E1
:100350009B928A827B746E68625C57524E4945411B
:100360003E3A3734312E2C29272523211F1D1C1AF4
:100370001917161514131211100F0E0D0C0B0A0974
:100380000807064500680100000500680138010003
:10039000000500380168010000A1039D030101FF71
:1003A000030101F70300000007000201000003043D
:1003B00006000000000000000001020408102040B8
:1003C0008001020408102001020408102004040423
:1003D00004040404040202020202020303030303EE
:1003E0000300000000230026002900000000002573
:1003F0000028002B0000000000240027002A000035
:100400006C0211241FBECFEFD8E0DEBFCDBF11E0DC
:10041000A0E0B1E0ECE2F2E302C005900D92A63656
:10042000B107D9F723E0A6E6B1E001C01D92AC3FC9
:10043000B207E1F712E0C1E0D2E004C02197FE016B
:100440000E94BF17C030D107C9F70E942B020C943D
:1004500014190C9400000E9466020E94C503FDCF8F
:100460000F931F93CF938C01C0E0F8018281C817CE
:1004700098F42C2F30E0C901880F991F322F2227C2
:10048000280F391F80819181820F931F009711F0EF
:100490000E94E802CF5FE9CF86E691E00E94450B1B
:1004A0008823D1F366E080E791E00E945704882317
:1004B000D9F242E064E770E086E691E00E94000C29
:1004C000813091F6CF911F910F9108950E940114F0
:1004D00086E691E00C94460F1092B7011092B60197
:1004E0008AE591E09093B5018093B4010895089551
:1004F0000895CF93DF93EC010E941F038EE391E0F8
:1005000099838883CE0188509F4F0E94640361E0E5
:1005100070E0CE014896DF91CF910C948A03BF9290
:10052000CF92DF92EF92FF920F931F93CF93DF93BF
:100530007C0102E011E0CEE1D1E0B12C6C0188EF4A
:10054000C80ED11C6B2D80E791E00E944E048823D9
:1005500071F1E881F9818A819B819C0121703327A7
:10056000309719F42115310589F095958795232B3E
:1005700051F0D701A80FB91F2D913C91E20FF31F45
:100580000190F081E02D8E0D9F1D0995D801ED9110
:10059000FC91119712968D919C911397309711F4BD
:1005A00080FF05C0959587958C0D9D1D0995B39489
:1005B0000C5F1F4F2496B7E0BB12C4CFDF91CF91E1
:1005C0001F910F91FF90EF90DF90CF90BF90089513
:1005D0000F931F93CF93DF93EC010E948F028E0144
:1005E000085E1F4FC850DF4FC8010E94BB03095F60
:1005F0001F4F0C171D07C1F7DF91CF911F910F916E
:100600000895FC01718360834283238314821582E1
:100610000895FC01648345830895CF93DF93EC0133
:100620006A8184EB91E00E944E05288139814D81D9
:100630006C8184EB91E0DF91CF910C943107AF9204
:10064000BF92CF92DF92EF92FF920F931F93CF93BF
:10065000DF93EC016B0184E491E0998388837E0150
:1006600088E0E80EF11C80E1F70111928A95E9F724
:100670008E01085E1F4F5E01F8EFAF0EB11C60E007
:1006800070E0C8010E947B03095F1F4F0A151B051C
:10069000B1F7C114D10431F040E150E0B601C70117
:1006A0000E94051943E050E06CE271E0CE01029631
:1006B000DF91CF911F910F91FF90EF90DF90CF903E
:1006C000BF90AF900C94FE18FC0110821282118230
:1006D00014821382168215821086178283E0818726
:1006E000089508950895FC011182108212821382E8
:1006F0001482089508950F931F93CF93DF93EC0115
:100700008B010E9473031E830D83DF91CF911F9194
:100710000F910895FC01768365830895CF93DF934D
:1007200000D000D000D0CDB7DEB7FC018581968126
:1007300083309105BCF4880F991FFC01E05BFE4FEC
:100740006081718120E041E0CE0101960E940103A9
:1007500040E160E1CE0101960E940903CE010196BD
:100760000E940D0326960FB6F894DEBF0FBECDBFD4
:10077000DF91CF910895CF93DF93EC010E947A032C
:10078000CE01DF91CF910C948E030F931F93CF93E3
:10079000DF93CDB7DEB7CF50D1400FB6F894DEBFB0
:1007A0000FBECDBF6AEA70E086E691E00E94C90EF6
:1007B00043E064EA70E086E691E00E94000C81115B
:1007C00024C08E010D5F1E4F8AE0F80111928A95B8
:1007D000E9F7B80186E691E00E94A10FB801025046
:1007E0001140C8010E94790281E0C15FDE4F888319
:1007F000CF50D140C35FDE4F19830883CD50D14025
:10080000CE01835F9E4F0E943002C15FDE4F0FB664
:10081000F894DEBF0FBECDBFDF91CF911F910F9136
:100820000895FC0188E0808389E0818387E08283EA
:1008300086E0838384E0848382E0858381E186830C
:100840000895FF920F931F93CF93DF93EC018C01D8
:10085000095F1F4FFF24FA9462E088810E94E1142F
:1008600088810E944C152F81892B19F42F5F2F83CB
:1008700007C0222349F02F3F11F41F8201C0FF82DD
:1008800060E088810E94E1142196C017D10721F70A
:10089000DF91CF911F910F91FF900895FC01E60F1A
:1008A000F11D81E09781913009F080E00895FC010D
:1008B000E60FF11D81E097819F3F09F080E00895E8
:1008C000262F30E0FC01E20FF31F423030F4978115
:1008D000915081E09E3F58F009C087818F3F31F0F1
:1008E000642F0E943F1781E0913009F080E0089565
:1008F0008EBD0DB407FEFDCF8EB50895DC016435C5
:1009000008F057C0403308F054C090969C919097DF
:10091000E42FE595E595E595262F062E000C330B83
:10092000542F57709230A1F4D90184E5E802A00D4C
:10093000B11D1124A351BE4F8C9190E0052E02C031
:10094000959587950A94E2F78095982F91700CC041
:10095000933051F41C968C916427062E000C770B73
:10096000682760FF03C014C0911112C084E5E8023B
:10097000200D311D1124F901E351FE4F81E090E07B
:1009800001C0880F5A95EAF780959081892310C09D
:1009900084E5E802200D311D1124F901E351FE4FD9
:1009A00081E090E001C0880F5A95EAF79081892B89
:1009B000808308951F93CF93DF93EC01162FF89453
:1009C00060E08F850E941D15888918161CF460E070
:1009D0000E941D15812F0E947804888918161CF426
:1009E00061E00E941D157894DF91CF911F910895C9
:1009F00028EF31E0EDEEF1E0DF01A9011D92415059
:100A00005040E1F7DC0119961C9219971A961C9236
:100A10000895CF92DF92EF92FF920F931F93CF939F
:100A2000DF93EC018C858F5F8C878DEEE82E81E063
:100A3000F82E10E0612F6064CE010E94DA0460E8B5
:100A4000CE010E94DA0461E08F850E941D1588891D
:100A500018161CF460E00E941D15670104E5F601FC
:100A600081916F010E9478040150C9F78889181696
:100A70001CF461E00E941D151F5FF4E5EF0EF11CF0
:100A80001630C1F660E4CE01DF91CF911F910F9136
:100A9000FF90EF90DF90CF900C94DA04FC0160A3FC
:100AA00061A30895FC0160A341A30895EF92FF9212
:100AB0000F931F93CF93DF938C01D62FF42EE22E4A
:100AC000C0E0CE1544F44F2D4C0F6D2FC8010E948D
:100AD0007E04CF5FF6CFDF91CF911F910F91FF90F2
:100AE000EF900895EF92FF920F931F93CF93DF93B0
:100AF0008C01F62ED42FE22EC0E0CE1544F46F2DDB
:100B00006C0F4D2FC8010E947E04CF5FF6CFDF919E
:100B1000CF911F910F91FF90EF900895DF92EF9288
:100B2000FF920F931F93CF93DF937C01D62FD22E8A
:100B3000C42F002E000C110B040F111D47FD1A9538
:100B40008C2F0C2E000C990B8017910744F42D2D3F
:100B50004C2F6D2FC7010E947205CF5FF1CFDF913F
:100B6000CF911F910F91FF90EF90DF9008958F929A
:100B70009F92AF92BF92CF92DF92EF92FF920F932C
:100B80001F93CF93DF937C01162FD42EC22F81E0C9
:100B9000C82EC21AB22EB194BB0CD0E0802F847044
:100BA000A82E802F8270982E802F8870882E01703A
:100BB000DC170CF04DC0C7FC04C0C150B394B39413
:100BC000CB0CDF5F8D2F880F8F5FC80EAA2071F0CE
:100BD0004D2D4C0F612F6D0FC7010E947E044D2DCE
:100BE0004D0F6C2F610FC7010E947E04992071F098
:100BF0004D2D4C1B612F6D0FC7010E947E044D2DA2
:100C00004D1B6C2F610FC7010E947E04882071F07C
:100C10004D2D4D0F612F6C1BC7010E947E044D2D81
:100C20004C0F612F6D1BC7010E947E04002309F445
:100C3000BFCF4D2D4D1B612F6C1BC7010E947E0441
:100C40004D2D4C1B612F6D1BC7010E947E04B0CF40
:100C5000DF91CF911F910F91FF90EF90DF90CF9098
:100C6000BF90AF909F908F9008958F929F92AF9278
:100C7000BF92CF92DF92EF92FF920F931F93CF9389
:100C8000DF936C01A62E942EC22F11E0121BF22EC0
:100C9000F194FF0C83E0B82EBE0CD1E0802F817060
:100CA000882EE39402708FEF8D0F8C17BCF517FD23
:100CB00004C0C150F394F3941F0D8D2F880F8F5FE4
:100CC000180F882091F02C2F220F2E0D492D4C1B30
:100CD0006D2F6A0DC6010E9456052B2D492D4D1B07
:100CE0006C2F6A0DC6010E945605011104C0DF5F1A
:100CF000B394B394D8CF2C2F220F2E0D492D4C1B1B
:100D00006A2D6D1BC6010E9456052B2D492D4D1BCA
:100D10006A2D6C1BC6010E945605E9CFDF91CF9169
:100D20001F910F91FF90EF90DF90CF90BF90AF9009
:100D30009F908F9008959F92AF92BF92CF92DF9233
:100D4000EF92FF920F931F93CF93DF936C01C62F07
:100D5000D42FB22EAE2CAA0C922E9A18FE2CF60E80
:100D6000292D6F2D0E9472051FEF100F1D0F292DC9
:100D7000412F6F2DC6010E9472050A19DE0D202F2A
:100D80004D2F6C2FC6010E945605CB0D6FEF6C0FD7
:100D9000202F4D2FC6010E94560501E02E2D4D2F0C
:100DA0006F2DC6010E94B7058E2D8095C80F02E0F9
:100DB0002E2D4D2F6C2FC6010E94B705D12FDE19A5
:100DC00004E02E2D4D2F6C2FC6010E94B70508E0C0
:100DD0002E2D4D2F6F2DC6010E94B705DF91CF91AB
:100DE0001F910F91FF90EF90DF90CF90BF90AF9049
:100DF0009F900895AF92BF92CF92DF92EF92FF92B1
:100E00000F931F93CF93DF936C01B62EF42E122F06
:100E1000C02FDE2DEE0CAD2EA60E2E196A2D0E94CF
:100E20008E05C150CE19FD0E6FEF6B0D610F6D1B5E
:100E3000EC2E01E02D2F4F2DC6010E94350602E059
:100E40002D2F4F2D6A2DC6010E943506DF91CF91BF
:100E50001F910F91FF90EF90DF90CF90BF90AF90D8
:100E600008952F923F925F926F927F928F929F92FE
:100E7000AF92BF92CF92DF92EF92FF920F931F93A8
:100E8000CF93DF93EC01F901E490319684916435BE
:100E90000CF019C10E2C000CFF08062F062E000CBA
:100EA000110BF701E00FF11F1E161F060CF00BC10E
:100EB00040330CF008C1A82FC42E042E000CDD080E
:100EC0005601A80EB11C87FDBA941A141B040CF02D
:100ED000FAC02E5F3F4F570197E0A90EB11CB7FE35
:100EE00004C05701BEE0AB0EB11CB3E0B594A794AB
:100EF000BA95E1F747FF0AC0A42FA80FAC9CC00128
:100F0000AD9C900D1124281B390B40E08A2F0A2E2E
:100F1000000C990B840F911D47FD9A95C19714F011
:100F2000A0E3A41BF8A067FD60E0E535F10514F02F
:100F3000E4E5F0E09E2FCC85C427C62E062E000CDB
:100F4000DD08F601E01BF10B8F014F01F7E08F2266
:100F50009924E0E8F0E002C0F595E7958A94E2F77D
:100F60007E2F17FF02C0095F1F4FF3E0159507950D
:100F7000FA95E1F7200F311F542F577081E001C01F
:100F8000880F5A95EAF7459545954595F601B4E5DC
:100F90004B02E00DF11D1124AF0143515E4FD0E033
:100FA0002A2EAA0F3308EE24E394BB24ED2FF0E0A1
:100FB000E215F3050CF087C0F9015490F1E0FF123F
:100FC0001AC0962E8A01E72F6901991608F072C09F
:100FD0008E2E852021F0D8018C90882A8C92E6955F
:100FE00031F4BFEFCB1ADB0AF6015490E0E893949A
:100FF0000F5F1F4FEACFF1101CC0782E7094962E11
:101000008A01E72F6901991608F054C08E2E8520B9
:1010100021F0D8018C9087208C92E69531F4BFEFB7
:10102000CB1ADB0AF6015490E0E893940F5F1F4F50
:10103000EACFF3E0FF1629F0962E8A01E72F690127
:1010400037C0682E6094862E8A01972E6901891612
:10105000D8F4E92DE52159F0D801EC917C2E7824C3
:1010600070FE02C0E82B02C0E621D801EC939694F2
:1010700039F4BFEFCB1ADB0AF6015490E0E89E2E5C
:1010800083940F5F1F4FE3CFCE2514C08E2E852093
:1010900021F0D8018C9088268C92E69531F4BFEF30
:1010A000CB1ADB0AF6015490E0E893940F5F1F4FD0
:1010B000991660F3880F19F44C5A5F4F81E0DF5F97
:1010C0002A0D3B1D73CFDF91CF911F910F91FF90A0
:1010D000EF90DF90CF90BF90AF909F908F907F90D8
:1010E0006F905F903F902F900895DC01FB018491F9
:1010F0008F5F14968C9314973196E491EF5F159659
:10110000EC9315976E5F7F4F5F967C936E935E971F
:101110000895EF920F93CF93DF93EC014E876D8785
:101120002F87E98A088B81E0888788A319A28F839B
:1011300069EB70E0CE010E9475080E94FC1681E008
:101140000E94121785E00E9420178CE00E941B1756
:1011500061E08E850E94E11461E08D850E94E114BA
:1011600061E08F850E94E114898918161CF461E002
:101170000E94E114888918161CF461E00E94E114B1
:10118000898918166CF460E00E941D156AE070E011
:1011900080E090E00E94DB1361E089890E941D15C8
:1011A0008D85082E000C990BFC01E353FC4FE49154
:1011B000F0E0EE0FFF1FE551FC4F259134913D8B80
:1011C0002C8BFC01E754FC4FE491EB8F8E85082EAD
:1011D000000C990BFC01E353FC4FE491F0E0EE0F9F
:1011E000FF1FE551FC4F259134913B8B2A8BFC016D
:1011F000E754FC4FE491EA8F8889082E000C990B84
:10120000FC01E353FC4FE491F0E0EE0FFF1FE551CA
:10121000FC4F259134913F8B2E8BFC01E754FC4F02
:10122000E491EC8F8F85082E000C990BFC01E353A1
:10123000FC4FE491F0E0EE0FFF1FE551FC4F2591CC
:101240003491398F288FFC01E754FC4FE491ED8FE6
:1012500061E2CE010E94DA0464E1CE010E94DA0468
:101260008B8587FF02C08FE78B876B856068CE0117
:101270000E94DA0460E2CE010E94DA046CE0CE0142
:101280000E94DA04CE01DF91CF910F91EF900C9480
:1012900009056F927F928F929F92AF92BF92CF92E9
:1012A000DF92EF92FF920F931F93CF93DF93EC01A6
:1012B00064350CF084C040330CF081C0EC81F0E068
:1012C00031970E9FC0010F9F900D1124860F911D25
:1012D00067FD9A95181619060CF071C03D81842F90
:1012E000042E000C990B039F800D911D11241816DC
:1012F00019060CF064C0D02EB42EC62E88A0A62EDF
:10130000962EE22EF12CEA2DEC190E2E000CFF0B7E
:101310008C8190E0E817F9070CF050C00197E817AE
:10132000F90779F0E89E9001E99E300DF89E300DA6
:101330001124E20FF31F8E8D9F8DE80FF91F14917A
:1013400001C010E07B2C6B2C272D2B19022E000CDA
:10135000330B8D8190E0281739076CF510FF11C011
:1013600081E0D81206C0472D6A2DCE010E947E046E
:101370001EC00D2D2D2D462D692DCE010E948E05EE
:1013800016C089A198A1891791F088A381E0D8128D
:1013900006C0472D6A2DCE010E947E0407C00D2D88
:1013A0002D2D462D692DCE010E948E0588A2169501
:1013B0006D0C7394C9CF9D0CA394A5CF88A2DF9127
:1013C000CF911F910F91FF90EF90DF90CF90BF9042
:1013D000AF909F908F907F906F9008950F93CF93D1
:1013E000DF93EC016A3011F428851EC06D3019F1CD
:1013F000262F08854A8569850E94490928853C81F0
:101400008985239F800D112489879F81992399F0D5
:10141000082E000C990B44E550E0239F4019510918
:101420001124481759073CF49D818A85299F800D16
:1014300011248A87198681E090E0DF91CF910F9186
:1014400008958F929F92AF92BF92CF92DF92EF92C8
:10145000FF920F931F93CF93DF93EC015C0186E81B
:10146000A80EB11CD5019C91992309F44DC09C3064
:1014700018F41CE0191B01C010E0FE01EA5AFF4FEE
:1014800081E080836E01BEE4CB0ED11C60E0C6011A
:101490000E944E054E01E3E58E0E911CD4018C9105
:1014A00003E0080F9DE2F92E4F2D481B410F23E06A
:1014B000E22E24E560E0C6010E94FA0661E0C60162
:1014C0000E944E05F401808103E0080F4F2D481B58
:1014D000410F24E560E0C6010E949B06FE01E95A27
:1014E000FF4F84E080833196D4018C91181B115DED
:1014F0001083CC57DF4F68817981C6010E94B215F5
:10150000F501808181508083DF91CF911F910F91F0
:10151000FF90EF90DF90CF90BF90AF909F908F9013
:101520000895CF92DF92FF920F931F93CF93DF9393
:10153000FC01248D358D232B09F49FC0EC018C0117
:10154000025B1F4F40E061E0C8010E945205FE01AE
:10155000E95AFF4FDE01AE5ABF4F9C9185E5891BCA
:10156000808331961082698D613009F463C028F060
:10157000888D653008F074C06FC0CE0185960E94DA
:10158000E71081E0FE01EA5AFF4F808369EB70E0CB
:10159000C8010E9475081D8E1C8EFE01EC5AFF4F7B
:1015A000108288EAF82E6E01FAE0CF0ED11CCE012F
:1015B0000E94450B8823D9F368EA72E0C8010E94B3
:1015C000B2156A8D7B8D4AE050E0C8010E94651615
:1015D00063E972E0C8010E94B2156F2D62956F70C9
:1015E00070E04AE050E0C8010E94B31668E872E07B
:1015F000C8010E94B21564E0C6010E944E04811128
:101600003CC0FA94F110D3CF60E0CE010E94BA1230
:1016100083B7817F846083BF83B7816083BF83B7D3
:10162000816083BF889583B78E7F83BF83B78E7FAA
:1016300083BFBDCFCF58DF4F88819981AA81BB81FD
:101640008F709927AA27BB270897A105B10510F429
:1016500067E009C068E707C0882379F06B5F03C0C3
:10166000882359F06FE2C801DF91CF911F910F914C
:10167000FF90DF90CF900C94D515DF91CF911F9103
:101680000F91FF90DF90CF9008958F929F92AF922D
:10169000BF92CF92DF92EF92FF920F931F93CF935F
:1016A000DF93EC017C0180E8E80EF11CF7018080FB
:1016B0009180A280B3800E94AA13861A970AA80A72
:1016C000B90A6E01FFE7CF0ED11CF601808190E0D0
:1016D000A0E0B0E08E0105581F4F88159905AA05B6
:1016E000BB0550F4F80180819181A281B381892BDF
:1016F0008A2B8B2B09F040C0F80180819181A28157
:10170000B381892B8A2B8B2BA9F57E01F5E2EF0E95
:10171000F11CC7010E94E410C7010E945011C701CB
:101720000E941512CE010E94210ACE010E94910A48
:101730007E018EE4E80EF11CC7010E940905FE013E
:10174000EC5AFF4F8081811103C0C7010E94F80449
:101750000E94B613F8016083718382839383FE0134
:10176000EB58FF4FC958DF4F28813981621B730B3B
:101770007183608380E037C00E94AA13F601208144
:10178000DC01CB01820F911DA11DB11DF7018083EA
:101790009183A283B383FE01EF58FF4F8081918133
:1017A000A281B3810196A11DB11D80839183A28383
:1017B000B383F80110821182128213820E94B61341
:1017C000FE01E958FF4F6083718382839383CE01CA
:1017D0000E94BE12CE010A960E942104CE014896B4
:1017E0000E94271381E0DF91CF911F910F91FF900D
:1017F000EF90DF90CF90BF90AF909F908F90089523
:101800002F923F924F925F926F927F928F929F9210
:10181000AF92BF92CF92DF92EF92FF920F931F93FE
:10182000CF93DF93CDB7DEB765970FB6F894DEBFE1
:101830000FBECDBF6C016A8B7B8B4B83FC01EC5AD6
:10184000FF4F10822FEF2D831C821D8A10E31C8A0C
:101850005C013AE0A30EB11C1C0183E5280E311C8B
:10186000BF972F01242F30E03F832E83C601895A72
:101870009F4F99878887F396FB87EA8796012A5AB4
:101880003F4F3F872E870297998B888B3A973F016E
:10189000C6010E94450B8823D9F364E0C5010E946C
:1018A0004E04012F110F110B811144C065E0C501D9
:1018B0000E944E0481113EC066E0C5010E944E04A4
:1018C000811138C02C8121114CC044E063E0C50176
:1018D0000E946004882331F03C893F5F3C8BC20149
:1018E0000E94921244E061E0C5010E9460048823D6
:1018F00031F08C8981508C8BC2010E949212EC894C
:101900008E2F0E2E000C990B2E813F81821793078C
:1019100031F0E7FF05C03B8131503C8B01C01C8A90
:10192000F1018081F4E0F80F2C89829FF0191124D5
:10193000FD8B22C0F101F081F98364E0C5010E94B2
:101940004E04882309F48CC0C2010E946612FC89EF
:10195000FD83298121953B81239F302D1124325015
:101960003D8BC8013D89831B910937FD93950297F3
:101970000CF47AC081E08C839D89090F111D97FDBD
:101980001A9517FF02C00F5F1F4FF801F595E795F5
:10199000FA83E9830981102FE885F9851082EA85A9
:1019A000FB85008381E0EE85FF858083E889F989E6
:1019B0001082EA88FB88812C912C2C89022E000C45
:1019C000330B3D872C878E819F818816990609F1FC
:1019D000EC85FD85E815F90579F423E0E885F985BE
:1019E0002083F1018081F02F2C89289FF00D112494
:1019F0008F2FEA85FB858083F70165917491C30180
:101A00000E94F015FFEF8F1A9F0A22E0E20EF11CF0
:101A1000DACF60E0C3010E944E05F1018081498167
:101A2000FC89F89F400D1124415024E560E0C3017A
:101A30000E94720561E0C3010E944E05F1018081A0
:101A400003E0080F4981FC89F89F400D11244250A2
:101A500083E0E82E24E560E0C3010E949B0618CFD6
:101A6000C2010E947C1275CF8D8165960FB6F894E5
:101A7000DEBF0FBECDBFDF91CF911F910F91FF90C1
:101A8000EF90DF90CF90BF90AF909F908F907F901E
:101A90006F905F904F903F902F9008950F931F93FA
:101AA000CF93DF93EC018C01025B1F4FC8010E94B2
:101AB000F80460E672E0C8010E94B215C8010E94F5
:101AC000090583E00E9420178EE591E0EEEFFFE329
:101AD0000995FE01EC5AFF4F10826BE372E0C801DA
:101AE0000E94F015C8010E9409052A96CE010E94A5
:101AF000210464E0CE010E944E04811107C062E31C
:101B000070E080E090E00E94DB13F0CFDF91CF9196
:101B10001F910F9108952F923F924F925F926F9273
:101B20007F928F929F92AF92BF92CF92DF92EF926D
:101B3000FF920F931F93CF93DF93CDB7DEB7299713
:101B40000FB6F894DEBF0FBECDBF3C0120E7620E9A
:101B5000711CF3012081222309F402C15A011B01E7
:101B6000998788877A9781E08083E885F985EB5AA1
:101B7000FF4F1082E885F985EC5AFF4F1082E88507
:101B8000F985108E8F01025B1F4F61E0C8010E9432
:101B90004E05888599858D5A9F4F9D838C83C88477
:101BA000D98497E5C90ED11CE884F984E8E5EE0EE6
:101BB000F11C888599858E5A9F4F9A838983E88581
:101BC000F985EF58FF4FFF83EE8388849984FAE00C
:101BD0008F0E911C4884598425E2420E511C888541
:101BE00099850E94450B8823D1F3F10184918823C4
:101BF00029F0EC81FD81F081FB8301C01B822AEC7E
:101C000032E040E060E0C8010E943107A114B10455
:101C100039F04B81445F950160E0C8010E943107B3
:101C2000F60110822CE0F7012083B101C8010E9467
:101C3000B215E981FA818081982F990F890F8195DA
:101C40008D5AF6018083EC81FD818081982F990F58
:101C5000890F8195835DF7018083EE81FF8180810B
:101C600084FF03C066EC72E002C062EC72E0C8015F
:101C70000E94F015E981FA818081982F990F890FD0
:101C800081958D5AF6018083F70180818F5F808373
:101C9000E885F98582A5882319F06EEB72E002C011
:101CA0006AEB72E0C8010E94F015E981FA81808137
:101CB000982F990F890F81958D5AF6018083F7012E
:101CC00080818F5F808366EB72E0C8010E94F0150F
:101CD00065E0C4010E944E04882351F0E885F9852F
:101CE00062A56F5FC2010E94A812C2010E949212F7
:101CF00064E0C4010E944E04811113C0F3012081ED
:101D0000422F50E060E070E0EE81FF8180819181A0
:101D1000A281B38184179507A607B707A8F02F3FC4
:101D200099F08FEFF3018083088519850B5D1F4FB4
:101D300060E0C8010E948510C8010E94661281E01F
:101D4000E885F985808F0CC066E0C4010E944E04CE
:101D5000882309F444CF888599850E944E0D35CF9C
:101D600029960FB6F894DEBF0FBECDBFDF91CF919D
:101D70001F910F91FF90EF90DF90CF90BF90AF90A9
:101D80009F908F907F906F905F904F903F902F909B
:101D9000089540E050E00C948B0DE0E8F7E72591C2
:101DA000349181E02130304C09F080E00895CF93E8
:101DB000DF93EC010E94CD0E9E01275A3F4FDE01BA
:101DC000A059BF4F882309F43CC0E6E9F7E78491A6
:101DD000F9018083E7E9F7E7E491EC83E8E9F7E7C5
:101DE000E491ED83E9E9F7E7859194919F838E83F0
:101DF000EBE9F7E78591949199878887EDE9F7E713
:101E0000E491EBA7EEE9F7E7E491EAA7EFE9F7E75A
:101E1000E491EC93E0EAF7E7859194919D8F8C8FA4
:101E2000E2EAF7E7859194919F8F8E8FE4EAF7E7D6
:101E30008591949199A388A3E6EAF7E78591949117
:101E400020C08CE3F90180831C828FEF8D8320E218
:101E500033E03F832E8324ED33E03987288791E0F8
:101E60009BA79AA78C938CEA9DE09D8F8C8F8EED1B
:101E70009DE09F8F8E8F84E79EE099A388A38CE3DB
:101E80009FE09BA38AA3DF91CF910895CF92DF9229
:101E9000EF920F93CF93DF93EC01FC01E158FF4FDA
:101EA00082E38083349781E090E0A0E0B0E080831B
:101EB0009183A283B3833B978FEF8083CE010E94EF
:101EC000D70ECE010E94B6126FEFCE010E94BA1259
:101ED0006E018AE0C80ED11CC6010E941104C60121
:101EE0000E942104CE0148960E941D138EE0E82E28
:101EF0000FE020E14BE06DE0CE01825B9F4F0E943E
:101F00008908A596CE010E94F10F65E0C6010E94E6
:101F10004E04882351F060E0CE01DF91CF910F9104
:101F2000EF90DF90CF900C94A81240E06AE373E04A
:101F3000CE01DF91CF910F91EF90DF90CF900C9475
:101F40009010CF93DF93D62FC72F0E94CD0E8823FA
:101F500059F0AD2FBC2FEBE8F7E784918D933196C4
:101F6000E53987E7F807C9F7DF91CF91089550E089
:101F7000DA01AA0FBB1FA80FB91F1F963C911F972C
:101F800050962C915097E32FF22FE60FF11DE60F9C
:101F9000F11D2591349190963C932E935F97F90112
:101FA00065917491FC017481769F602D1124DC0190
:101FB000A40FB51F91966C939197F9018591949117
:101FC000E92FF0E0862F90E0E817F90720F4F901F7
:101FD00085919491692F769F602D112492966C9330
:101FE000089521E0FC01248324E020A729E933E0BF
:101FF000308B278740E060E00E94B70F61E070E01F
:1020000083E00E945914E1EBF0E08081887F8160D9
:102010008083F89410928000E1E8F0E01082109242
:1020200085001092840088E191E09093890080936C
:102030008800808188608083808181608083EFE672
:10204000F0E0808182608083789408950F93FC0192
:10205000842F01112AC06230D9F050F4662399F020
:10206000613019F540E0682FCF010F910C94B70F44
:102070006330A9F06430C9F46481649F802D112419
:10208000858F268F12C04B3008F08AE0868B0DC0FA
:102090006481649F802D1124818F228F06C064810A
:1020A000649F802D1124838F248F0F910895FC014C
:1020B00021110EC0648B8481849F402D1124458B97
:1020C00015A214A213A281E0878B8093F103108ED6
:1020D00008958091F103882319F08091EE0301C0E7
:1020E00080E08093B4000895FC0161110DC0178A4F
:1020F000158A14A213A2108E1092EE031092EF0311
:102100001092F1030C9469100895CF93DF9361113D
:1021100004C0EC010E9474101982DF91CF910895E0
:102120000F931F93CF93DF93411110C08B01EC01EC
:1021300060E00E9485101E870D871B8A1A8A81E045
:10214000898389E08E8B198E1B8E1D8EDF91CF9136
:102150001F910F910895CF93DF93DC01611131C07E
:102160008C91882371F111968C911197811129C05E
:1021700019968C91199717962C91179718969C91F0
:102180001897E22FF92FE80FF11DE80FF11D2591A7
:1021900034912F3F8FEF380711F41C9212C0ED01DC
:1021A0003C873327220F331FEA85FB85E20FF31F9D
:1021B0006591749140E0CD010E94901089858F5FF8
:1021C0008987DF91CF91089560E00C94AB1060E0B7
:1021D0000C9485100F93CF93DF93EC0161115CC0D9
:1021E0008981882309F458C08D89811155C02D85B6
:1021F0003E85EA89FB89EE0FFF1FE20FF31F8591F1
:102200009491009701F58989813021F41B8A1A8AFB
:10221000F90110C01982888160E0882371F0CE0135
:102220000E94AB10EA89FB89EE0FFF1F8D859E850A
:10223000E80FF91F8591949106C0CE01DF91CF91EF
:102240000F910C947410BC017695679576956795FF
:1022500080FF17C0AC0186E0569547958A95E1F757
:10226000292F26952695269520514F716F7000E0F5
:10227000CE010E942610EA89FB893196FB8BEA8BFE
:10228000D3CF492F6F7320E0CE010E9457108A8967
:102290009B8901969B8B8A8BDF91CF910F9108953B
:1022A00060E00C94EA10CF93DF93EC016111BAC0A7
:1022B0008F89882309F4B6C09D89911105C0CE018C
:1022C000DF91CF910C94741091509D8B8DA1811151
:1022D00039C02BA13CA12F5F3F4FC901880F991F27
:1022E000EF8DF8A1E80FF91F65917491862F877023
:1022F0008EA3AB0163E0569547956A95E1F7CA0155
:1023000096958795972F969596959FA38F739C8109
:10231000899F802D11248DA341704093ED033CA330
:102320002BA389A190E02817390760F02AA1222366
:1023300029F0821B91099CA38BA304C060E0CE010D
:102340000E9474108DA181508DA3888D21E0280FEB
:10235000288F4C893FA1340F8C85380F3A836B8DC1
:10236000662361F070E0822F022E000C990B0E9410
:102370005F178C8D869F300D11243A838A8190E0FF
:10238000CB966BE370E00E945F178A833E893B83A4
:10239000698D662371F0062E000C770B822F022EBA
:1023A000000C990B0E945F178A8D869F300D1124B7
:1023B0003B836D8D662389F0822F220F990B70E08D
:1023C0000E945F17CB0162E070E00E945F172E8DC4
:1023D0009B81289F900D11249B834F3341F08B816B
:1023E0008A300CF089E087FD80E08B8301C01B827E
:1023F000F894EA81F0E0E85BFC4FE491E093F003AD
:102400008D8198A5899F802D11249B81899F802D86
:1024100011249EA1899F802D11248093EF03809326
:10242000EE037894DF91CF91089560E00C945311FE
:102430006091EF03662329F18091F2038F5F80930F
:10244000F2039091F0038917E0F081E09091F1039D
:10245000911180E08093F1031092F2038091ED03DB
:10246000882369F08091000193E4899F802D1124D5
:10247000895B809300010E943F179093EE030C94B8
:10248000691008951F920F920FB60F9211242F9387
:102490003F934F935F936F937F938F939F93AF93EC
:1024A000BF93EF93FF930E941812FF91EF91BF919A
:1024B000AF919F918F917F916F915F914F913F91DC
:1024C0002F910F900FBE0F901F901895CF93DF9311
:1024D000EC0160E00E94851081E993E09E878D8782
:1024E0001B8A1A8A81E0898389E08E8B198E1B8E64
:1024F0001D8EDF91CF910895CF93DF93EC0160E0C3
:102500000E94851089E893E09E878D871B8A1A8A2E
:1025100081E0898389E08E8B198E1B8E1D8EDF9161
:10252000CF910895CF93DF93EC0160E00E94851076
:1025300083E893E09E878D871B8A1A8A81E08983CE
:1025400089E08E8B198E1B8E1D8EDF91CF910895A1
:10255000FC01262F660F330B9681692F70E06F5FA9
:102560007F4FC9010E945F178583089521E0FC0118
:102570002083089570E085E00C945914AF92BF92C7
:10258000CF92DF92EF92FF920F931F93CF93DF933F
:10259000EC0189819A812FE0289F8001299F100DED
:1025A000112485E10E943C14800F911F24E0969530
:1025B00087952A95E1F79A8389832881222391F1CF
:1025C000EC81AD80B12CC12CD12CA885B9857D01C1
:1025D00000E010E06E817F819B0140E050E08617B3
:1025E000970728F0BC01A817B90708F4BD0180E0DF
:1025F00090E01F921F921F92EF930E94BA166B8376
:102600000F900F900F900F9070E085E0DF91CF91C9
:102610001F910F91FF90EF90DF90CF90BF90AF9000
:102620000C945914DF91CF911F910F91FF90EF906F
:10263000DF90CF90BF90AF900895FC018CE39FE0B6
:102640009383828384E0818381E084870895CF939C
:10265000DF93FC0124813581232B79F1EC01848502
:102660008F7141F584E10E943C14BC01990F880BE5
:10267000990B0E94051826EE3FE34EEC50E40E94B1
:1026800091180E94D4179B017B836A83672B81F08A
:1026900084E08983FE01349680E0419151912417B2
:1026A000350710F4898309C08F5F8430B1F702C009
:1026B0008FEF89838C858F5F8C87DF91CF91089511
:1026C0001F920F920FB60F9211242F933F938F9367
:1026D0009F93AF93BF938091F4039091F503A091E2
:1026E000F603B091F7033091F30323E0230F2D3766
:1026F00020F40196A11DB11D05C026E8230F029606
:10270000A11DB11D2093F3038093F4039093F5036F
:10271000A093F603B093F7038091F8039091F90327
:10272000A091FA03B091FB030196A11DB11D809306
:10273000F8039093F903A093FA03B093FB03BF91BE
:10274000AF919F918F913F912F910F900FBE0F905E
:102750001F9018952FB7F8946091F4037091F503CA
:102760008091F6039091F7032FBF08953FB7F89437
:102770008091F8039091F903A091FA03B091FB03C3
:1027800026B5A89B05C02F3F19F00196A11DB11DCC
:102790003FBFBA2FA92F982F8827820F911DA11D07
:1027A000B11DBC01CD0142E0660F771F881F991F44
:1027B0004A95D1F70895CF92DF92EF92FF92CF938F
:1027C000DF936B017C010E94B613EB01C114D104AD
:1027D000E104F10479F00E94B6136C1B7D0B683E96
:1027E0007340A0F381E0C81AD108E108F108C8518C
:1027F000DC4FECCFDF91CF91FF90EF90DF90CF9047
:102800000895789484B5826084BD84B5816084BD68
:1028100085B5826085BD85B5816085BDEEE6F0E059
:10282000808181608083E1E8F0E0108280818260B5
:102830008083808181608083E0E8F0E08081816036
:102840008083E1EBF0E0808184608083E0EBF0E066
:10285000808181608083EAE7F0E08081846080830A
:1028600080818260808380818160808380818068B4
:1028700080831092C10008958E3008F08E50209110
:10288000010190E4299F900111248770822B80938D
:102890007C0080917A00806480937A0080917A0035
:1028A00086FDFCCF809178002091790090E0922BFA
:1028B00008951F93CF93DF93182FEB0161E00E94DF
:1028C000E114209711F460E004C0CF3FD10539F442
:1028D00061E0812FDF91CF911F910C941D15E12FA5
:1028E000F0E0EB55FC4FE491E330F9F048F4E130CF
:1028F000B9F0E230A1F584B5806284BDC8BD34C0B2
:10290000E630E9F0E73019F1E43049F580918000D4
:10291000806280938000D0938B00C0938A0024C093
:1029200084B5806884BDC7BD1FC080918000806869
:1029300080938000D0938900C093880015C0809157
:10294000B00080688093B000C093B3000DC0809148
:10295000B00080628093B000C093B40005C0C0385E
:10296000D1050CF0B5CFAFCFDF91CF911F91089576
:10297000833081F028F4813099F08230A1F00895FD
:102980008630A9F08730B9F08430D1F4809180008E
:102990008F7D03C0809180008F77809380000895A1
:1029A00084B58F7702C084B58F7D84BD08958091F2
:1029B000B0008F7703C08091B0008F7D8093B0000E
:1029C0000895CF93DF9390E0FC01E754FC4F2491EE
:1029D000FC01E353FC4F8491882361F190E0880F60
:1029E000991FFC01EB50FC4FC591D491FC01E551BE
:1029F000FC4FA591B491611109C09FB7F8948881EB
:102A0000209582238883EC912E230BC0623061F4E1
:102A10009FB7F8948881322F309583238883EC9177
:102A20002E2B2C939FBF06C08FB7F894E8812E2BD6
:102A300028838FBFDF91CF9108951F93CF93DF93AA
:102A4000282F30E0F901EB55FC4F8491F901E75450
:102A5000FC4FD491F901E353FC4FC491CC23C1F056
:102A6000162F81110E94B814EC2FF0E0EE0FFF1F1B
:102A7000E551FC4FA591B4919FB7F894111104C092
:102A80008C91D095D82302C0EC91DE2BDC939FBFB4
:102A9000DF91CF911F910895CF93DF93282F30E0DE
:102AA000F901EB55FC4F8491F901E754FC4FD491A7
:102AB000F901E353FC4FC491CC2391F081110E94A2
:102AC000B814EC2FF0E0EE0FFF1FEF51FC4FA59173
:102AD000B491EC91ED2381E090E021F480E002C01C
:102AE00080E090E0DF91CF910895CF92DF92EF9256
:102AF000FF920F931F93CF93DF936C01EB017B0148
:102B0000E40EF51E00E010E0CE15DF0561F06991DE
:102B1000D601ED91FC910190F081E02DC60109955F
:102B2000080F191FF1CFC801DF91CF911F910F91AD
:102B3000FF90EF90DF90CF9008956115710579F0C7
:102B4000FB0101900020E9F73197AF01461B570BBD
:102B5000DC01ED91FC910280F381E02D099480E08D
:102B600090E00895EF92FF920F931F93CF93DF931E
:102B70007C01FB0100E010E06491EF0121966623E7
:102B800061F0D701ED91FC910190F081E02DC7013A
:102B90000995080F191FFE01EFCFC801DF91CF91F2
:102BA0001F910F91FF90EF900895DC01ED91FC9142
:102BB0000190F081E02D09940F931F93CF93DF9341
:102BC000EC016DE00E94D5158C016AE0CE010E94F7
:102BD000D515800F911FDF91CF911F910F9108950F
:102BE0000F931F93CF93DF93EC010E94B2158C01DA
:102BF000CE010E94DC15800F911FDF91CF911F91B4
:102C00000F9108958F929F92AF92BF92CF92DF92D1
:102C1000EF92FF920F931F93CF93DF93CDB7DEB761
:102C2000A1970FB6F894DEBF0FBECDBF6C01142F75
:102C3000E52FCB01022F19A2223008F40AE07E0111
:102C400021E2E20EF11C802E912CA12CB12C612FDF
:102C50007E2FA50194010E947317029F1019112461
:102C600081E0E81AF1081A3014F4105D01C0195C13
:102C7000F7011083122FE32FCA01232B242B252BBE
:102C800031F7B701C6010E949D15A1960FB6F894C1
:102C9000DEBF0FBECDBFDF91CF911F910F91FF908F
:102CA000EF90DF90CF90BF90AF909F908F9008955E
:102CB0002115310541F4DC01ED91FC910190F08189
:102CC000E02D642F09940C9402169A01AB0160E088
:102CD00070E00C945816CF92DF92EF92FF920F9310
:102CE0001F93CF93DF932115310581F4DC01ED9122
:102CF000FC910190F081E02D642FDF91CF911F9125
:102D00000F91FF90EF90DF90CF9009942A3031051A
:102D100001F577FF1DC06A017B01EC016DE20E94A5
:102D2000D5158C0144275527BA014C195D096E0948
:102D30007F092AE0CE010E940216800F911FDF91C9
:102D4000CF911F910F91FF90EF90DF90CF9008955A
:102D50002AE0DF91CF911F910F91FF90EF90DF90CC
:102D6000CF900C9402169A01AB01770F660B770B8C
:102D70000C946B164F925F926F927F92AF92BF92BC
:102D8000CF92DF92EF92FF920F931F93CF93DF9337
:102D9000CDB7DEB729013A019B01AC0124193509F1
:102DA0004609570989899A89AB89BC89BC01CD013B
:102DB0006A197B098C099D090E942F17A8019701A8
:102DC00024193509460957090E949517CA01B90106
:102DD0006A0D7B1D8C1D9D1DDF91CF911F910F9161
:102DE000FF90EF90DF90CF90BF90AF907F906F906B
:102DF0005F904F900895089561E08AE00E941D154C
:102E000061E08AE00E94E1148CB580618CBD8CB5D4
:102E100080648CBD61E08DE00E94E11461E08BE094
:102E20000C94E114811103C08CB5806202C08CB592
:102E30008F7D8CBD08959CB5937F892B8CBD0895A3
:102E40009CB59C7F282F2370922B9CBD2DB582FBB7
:102E5000992790F9822F8E7F892B8DBD0895DB01F4
:102E60008F939F930E94B417BF91AF91A29F800D43
:102E7000911DA39F900DB29F900D11240895991B51
:102E800079E004C0991F961708F0961B881F7A9561
:102E9000C9F780950895AA1BBB1B51E107C0AA1F63
:102EA000BB1FA617B70710F0A61BB70B881F991FEB
:102EB0005A95A9F780959095BC01CD01089597FB8F
:102EC000072E16F4009407D077FD09D00E944B1707
:102ED00007FC05D03EF4909581959F4F089570951D
:102EE00061957F4F0895A1E21A2EAA1BBB1BFD011D
:102EF0000DC0AA1FBB1FEE1FFF1FA217B307E407D9
:102F0000F50720F0A21BB30BE40BF50B661F771F30
:102F1000881F991F1A9469F7609570958095909510
:102F20009B01AC01BD01CF010895052E97FB1EF456
:102F300000940E94AC1757FD07D00E94731707FC3E
:102F400003D04EF40C94AC175095409530952195D4
:102F50003F4F4F4F5F4F08959095809570956195C5
:102F60007F4F8F4F9F4F08950E94C517A59F900DCB
:102F7000B49F900DA49F800D911D11240895EE0F14
:102F8000FF1F0590F491E02D0994A29FB001B39F1B
:102F9000C001A39F700D811D1124911DB29F700D62
:102FA000811D1124911D08950E94701888F09F576B
:102FB00098F0B92F9927B751B0F0E1F0660F771F5D
:102FC000881F991F1AF0BA95C9F714C0B13091F053
:102FD0000E948A18B1E008950C948A18672F782F00
:102FE0008827B85F39F0B93FCCF386957795679518
:102FF000B395D9F73EF490958095709561957F4F84
:103000008F4F9F4F0895E89409C097FB3EF4909529
:103010008095709561957F4F8F4F9F4F9923A9F0B1
:10302000F92F96E9BB279395F69587957795679540
:10303000B795F111F8CFFAF4BB0F11F460FF1BC084
:103040006F5F7F4F8F4F9F4F16C0882311F096E917
:1030500011C0772321F09EE8872F762F05C06623C5
:1030600071F096E8862F70E060E02AF09A95660F7E
:10307000771F881FDAF7880F9695879597F9089537
:1030800097F99F6780E870E060E008959FEF80EC1B
:10309000089500240A9416161706180609060895BE
:1030A00000240A9412161306140605060895092E24
:1030B0000394000C11F4882352F0BB0F40F4BF2B93
:1030C00011F460FF04C06F5F7F4F8F4F9F4F0895D3
:1030D00057FD9058440F551F59F05F3F71F04795C9
:1030E000880F97FB991F61F09F3F79F087950895AE
:1030F000121613061406551FF2CF4695F1DF08C0CD
:10310000161617061806991FF1CF869571056105E9
:1031100008940895E894BB2766277727CB0197F991
:1031200008950E94A4180C9457180E94491838F06A
:103130000E94501820F0952311F00C9440180C9424
:10314000461811240C948B180E94681870F3959FF0
:10315000C1F3950F50E0551F629FF001729FBB278E
:10316000F00DB11D639FAA27F00DB11DAA1F649F2A
:103170006627B00DA11D661F829F2227B00DA11DDD
:10318000621F739FB00DA11D621F839FA00D611D63
:10319000221F749F3327A00D611D231F849F600D84
:1031A000211D822F762F6A2F11249F5750409AF0AD
:1031B000F1F088234AF0EE0FFF1FBB1F661F771F39
:1031C000881F91505040A9F79E3F510580F00C9404
:1031D00040180C948B185F3FE4F3983ED4F3869527
:1031E00077956795B795F795E7959F5FC1F7FE2BA4
:1031F000880F911D9695879597F90895DC0101C078
:103200006D9341505040E0F70895FB01DC014150BF
:10321000504048F001900D920020C9F701C01D9266
:0C32200041505040E0F70895F894FFCFB3
:10322C0001017103000000000000720300000000A7
:10323C000000000000000000000000000000000082
:10324C0000000000000000000000000000007802F8
:10325C000000770200000000000000000000770270
:10326C0000000000FB160808003C4299A5661800F7
:10327C0000004601000000000000EE0975154C4FDF
:06328C0041444552000020
:04000003000004569F
:00000001FF
